:030000000219FDE5
:03000B000200A848
:03002B000201636C
:03005B000202EDB1
:030073000202D3B3
:1000800002030406080C10182030406080040608A3
:100090000C10182030406080A0C000070F1F3F05E3
:1000A000050D050305030302C2AFC0D0C0E0206206
:1000B00017E5256002E473E525F4F58A758B00D217
:1000C00062D0E0D0D0D2AF3285268AC262E526F473
:1000D0006035306803207210758B00D0E0D0D0D22C
:1000E00092D291D290D2AF32D292D291D290206E4F
:1000F0000C206609740AD5E0FDE57E4290758B0000
:10010000D0E0D0D0D2AF32758A00C28DD26201FD6C
:1001100001B7306805206602C29201B73068052039
:100120006602C29101B7306805206602C29001B72D
:10013000C29330680A2066077408D5E0FDC29201B8
:10014000B7C29430680A2066077408D5E0FDC291F2
:1001500001B7C29530680A2066077408D5E0FDC271
:100160009001B7C2AFC2AD53E6EFC0D0C0E0D2D36A
:10017000D2AFC2CEE52A6007207449152A21C4787F
:1001800000790020742EE580307E01F430E402789E
:10019000FF53DACF207E0343DA20307E0343DA10A8
:1001A000C2D8C271E580307E01F430E40279FFC329
:1001B000E89970CB306103752A18207403752A18EA
:1001C000885FD27020740DE52B6004152B21D44379
:1001D000DA01C2D82070024136A85F206102C270E5
:1001E000207431C3E894F0400374F0F8E8C4540F6D
:1001F00028F87984B703024114C313C3138721205D
:100200000802C313200A06C3C898F8411428F850FE
:100210000374FFF8C3E895685003E568F88822E5A1
:100220002D54066011E533C313C31324062522F5AC
:100230002250037522FF852224A824C3E524956457
:100240004002A8648825E5697002417AC3E8AA697A
:100250009A5003E8FAE4F9EAC333FBE56BF45B294F
:10026000400D256AF8E56A6002156A400B417A0A7A
:10027000C3E56A9A5002056A78FF8826C26EC3E514
:100280002694F84002D26EC3E52594404002D26421
:1002900020CF0AD0E0D0D043E610D2AD32C2CF0595
:1002A0003A7801E52A6005307402152AC3E55F94A7
:1002B00001400575620041C9756300756C00E56217
:1002C0002401F56250037562FFD0E0D0D043E61000
:1002D000D2AD32C2AFC0D053E67FC2607591008507
:1002E0005694855795759104D0D0D2AF32C2AF5392
:1002F000E6EFC2ADC0D0C0E0C0F0D2D3D2AFA8FB11
:10030000A9FCC2D8307102615453DACF207E034376
:10031000DA10307E0343DA20D271E580307E01F4BA
:1003200020E402612B88278928A17B53DACF207E25
:100330000343DA20307E0343DA10C2D8C27130742E
:1003400002A1677800E580307E01F430E402A16705
:10035000885FA14F53DACF207E0343DA20307E033B
:1003600043DA10C271206102812D53DACF207E035F
:1003700043DA10307E0343DA20C2D8D271885A891A
:100380005BC3E89558F8E99559F97B007E087A0037
:10039000C3E8948CE994005005755E00811F8821A4
:1003A00078A2E6A8216055C3E894C8E994005008F3
:1003B000E4D2E4FB7A0A61FAC3E89468E994015054
:1003C00008E4D2E3FB7A0F61FAC3E894D0E994021F
:1003D0005008E4D2E2FB7A1E61FAC3E894A0E994E3
:1003E000055008E4D2E1FB7A3C61FAC3E89498E94D
:1003F00094085008E4D2E0FB7A787E00C3E8955C6C
:10040000FCE9955DFD30E70AECF42401FCEDF434E1
:1004100000FD755E00C3EC9AED9E5003755E018889
:100420005C895D855A58855B597802A14FC3E89570
:1004300027F8E99528F9307C02A133307B02A133FB
:10044000307A02A12C2075028150E9FDE8FC816F11
:10045000E9C313F9E813F8307902A12CE9C313F9C1
:10046000E813F8307802A12CE9C313FDE813FC204F
:0E0470006126C3EC941CED940240028186EDDF
:10047E007018C3EC94C850120529C3E529940A508C
:10048E0002A167755F00D270A167E5296002152988
:10049E007888E6F97400207F087896B90302789E72
:1004AE00E624FAFEE43400FFC3EC9EFCED9FFD92C1
:1004BE0008B90310A2085007207609D27681D230EF
:1004CE007602C276A2085016B9030DECF42401FC94
:1004DE00EDF43400FD0204EC78007900A133B90389
:1004EE0015EC33FCED33FDC3EC940AFCED9400FDEA
:1004FE0050047C007D00C3EC94FFED940040067820
:10050E00FF7900A133EC8575F0A4C5F0A2F733F89E
:10051E007900400302054F78FF790002054FE9C3C9
:10052E0013F9E813F8307C0EE9600278FFC3E81384
:10053E0038F8E43400F9C3E894FFE99400400278F7
:10054E00FF885FD270206102A167741FF4552F4B94
:10055E00F52FC274EB7002D274752A1830740375BD
:10056E002A0A306102A17B20740353DAFE20740341
:10057E00752B06D0F0D0E0D0D0D2AD43E610327954
:10058E00010205AB79030205AB790A0205AB791EB0
:10059E000205AB79640205AB79C80205AB7817E4A6
:1005AE00D5E0FDD8FAD9F6227A147B780205D27AF4
:1005BE00107B8C0205D27A0D7BB40205D27A0B7BAE
:1005CE00C80205D27902B27DE4C294D5E0FDC29193
:1005DE00D5E0FDD291D5E0FDD294D5E0FDC292E5F5
:1005EE0076D5E0FDD2927496D5E0FDD9D9EAF8D54C
:1005FE00E0FDD8FBDBCEC29422C37C007D0075F0FB
:10060E000005F0EA33FAEB33FB50F6EB13FBEA137B
:10061E00FAC3E9FFE8FEE89AF8E99BF95004EFF90E
:10062E00EEF8B3EC33FCED33FDD5F0DFEDF9ECF87D
:10063E0022E889F08A20D2D4F8A9F07B0030F70B9B
:10064E007BFFF42401F8E9F43400F9E88520F0A4E6
:10065E00ADF0F8E98520F0A4AFF0FEED2EF97400B0
:10066E003FFA7C04C3EA13FAE913F9E813F8DCF451
:10067E008BF030F70AE8F42401F8E9F43400F9E8D5
:10068E0089F0C2D4F8A9F02222C3E54113F9E5405E
:10069E0013F8C3E54598F8E54699F9500CC3E8946C
:1006AE0080E994FF40160206CEC3E8947FE99400D9
:1006BE0050030206CE787F79000206CE788079FF4D
:1006CE00884A894B22E54A2547F8E54B3548F98596
:1006DE004B20E4300701F43549FA30E709C3EA94B8
:1006EE00F0401502070CC3EA940F500302070C7872
:1006FE00FF79FF7A0F02070C780079007AF0C3E5D4
:10070E00249564500AC374019524500B02072AE500
:10071E004B20E70E02072AE54B30E706884789484B
:10072E008A492278A4E6FAC3E54A33F8E54B33F951
:10073E00D13FE930E70BC3E89480E994FF4013E121
:10074E0064C3E8947FE994005002E164787F7900F5
:10075E00E164788079FFE820E715C3E52398F84037
:10076E0009C3E89401400302078B780102078BE866
:10077E00F424012523F8400302078B78FF884C22CE
:10078E0078A5E6FAA848A949D13FE930E70CC3E8B5
:10079E009401E994FF40160207BFC3E894FFE99461
:1007AE000050030207BF78FF79000207BF78017976
:1007BE00FFE920E715C3E54C98F84009C3E894011A
:1007CE0040030207E678010207E6E8F42401254C0F
:1007DE00F840030207E678FF88242278FFC26420DF
:1007EE00693D206A12D264C3E541940A4009C3E50B
:1007FE002594405002C26479A1E76023E541601F51
:10080E0074FF8541F0848539F0306A0375F005A4D4
:10081E00F8C5F0600278FFC3E895675002A86788B4
:10082E006622C3E5409440E5419401E56650031409
:10083E000141046002F566220208492275E8902201
:10084E007883E6FFE5E820ECF7A8BDA9BE0573C3E3
:10085E00E57394084052757300E9FA79A0E7604495
:0E086E00EA7007E574601B020884C3E8957405
:10087C006010E5745006600C140208900460F902D4
:10088C000890E574F574C39458401B7564C0C39408
:10089C00044013756480C39404400B756440C39486
:1008AC0004400375640075BB0322E564F460020523
:1008BC0064E573B4070375BB1022743279A687F014
:1008CC00A4C5F0A2F733F8C3E895644002A8648885
:1008DC00228824882588268867227540007541F077
:1008EC0022C2AF75C820A8CCA9CDAA3A30CF010A34
:1008FC0075C824D2AFAB3BAC3C883B893CC3E89B6E
:10090C00F8E99C206908F93067024102215FAD3D8E
:10091C008A3DF9EA9DFA600478FF79FFAE3EAF3F5D
:10092C008B3E8C3FC3EC9FFCC3E99CF542A83BA9D2
:10093C003CC3E89EF8E99FF9C3E54113FBE540137E
:10094C00FAE82AF540E93BF54150067540FF754140
:10095C00FF21A9AA40AB41AC40AD417E047F02C34C
:10096C00EB940440021E1FC3EB940840021E1FC3ED
:10097C00ED13FDEC13FCDEF7C3EA9CFAEB9DFBEFE9
:10098C006009C3E913F9E813F8DFF7EA28FAEB3941
:10099C00FB8A408B4150067BFF8B408B41C3EB9411
:1009AC00025002D2673069047F0321D47892E6FFAB
:1009BC00C3E537948240110FC3E53794A040010F73
:1009CC00C3EF940640027F057E05E541C4540FF940
:1009DC00E541C454F0F8E540C4540F28F8C3E89E30
:1009EC00FAE99400FB4009C3EA9402EB940050042A
:1009FC007A02E4FB414EAA40AB41EBC4FEEAC4547C
:100A0C000F4EFCC3EA9CFAEB9400FBC3E813C31330
:100A1C00F8EA28FAEB3400FB8A408B41C3EB9402D2
:100A2C004002C2677805EBC4FE7B00EAC4540F4E4B
:100A3C00FAC3EA98FA4005C3940250027A027892FB
:100A4C00E6FF306002414E855256855357D26043C3
:100A5C00E680C3E49AF8E49BF930670241E8E8FACF
:100A6C00E9FBD3E913FDE813FC88528953C3EF94D7
:100A7C00036038EF20E00DE82CF8E93DF9ECFAEDD5
:100A8C00FB020AA3E828F8E939F9C3E82402F8E9DB
:100A9C003400F97AFE7BFFC3EF9403400E8A548B2B
:100AAC0055884E894F8C508D51611C885489558ABC
:100ABC004E8B4F8C508D51306920C3E533940340DD
:100ACC0019E542A2E713F8E555F4240138400B2050
:100ADC00E7087554FFF42401F555611CE8FAD3E8D6
:100AEC0013FC8852C3EF94036020EF20E007E82C3E
:100AFC00F8ECFA6108E8282402F87AFEC3EF9403B4
:100B0C0040088A54884E8C50611C88548A4E8C50F4
:100B1C00E56BC3335002646BF56B30600261267574
:100B2C003402D26043E680E52D54066026A840A925
:100B3C0041C3E913F9E813F8C2AF53E67F7591008E
:100B4C00C3E498F594E499F595759104D26043E665
:100B5C0080D2AF22D265754400752000306B0375CE
:100B6C002040020B7FD265754400752040306B032A
:100B7C00752000D2AF7801206722E52D5406600263
:100B8C00C265C3E54194054013780294054008788A
:100B9C0003940540027806306902780A206019E552
:100BAC0044601530690AC3E53394034003D5340619
:100BBC00D2AFD26C8151712ED2AF0000C2AF206780
:100BCC0026E541C3FB940F40027B0FEB24053073E9
:100BDC000123306A02742820620123F930690279FA
:100BEC0082E58BC39940B50544E59BF45440B52090
:100BFC0002813B30690A08C3E8940A40010861A8E5
:100C0C00206502617FC26553E67F759100306710E5
:100C1C007594007595FE759104D26043E680617FF2
:100C2C00AE40AF41C3E49EF594E49FF5958122C399
:100C3C00E53394025002617F306502617FD80281F6
:100C4C004F61A8C26C53E67F75910085549485550D
:100C5C0095759104854E56854F57D26043E680D2E8
:0F0C6C00AFE52D54066008206A020533020C8B99
:100C7B00306C0D206B0A2065071581158102151A42
:100C8B002278003064053065027801E53775F0078E
:100C9B00A4F9E5F028F5F0E9A2F013A2F113A2F202
:100CAB0013F537C394785003753778C3E537953808
:100CBB004008D266D292D291D29030600281C58523
:100CCB005056855157D26043E68022D2A0207D1129
:100CDB00C2AF754302C294D293D2AF759F10020E6E
:100CEB00B1C2AF754302C294D295D2AF759F1002B9
:100CFB000EB1C2A0307243207D20C2AF754303906A
:100D0B000141757E10D290C295306204C291A11D33
:100D1B00D294D2AF759F20020EB1C2AF7543039030
:100D2B000141757E10D292C293306204C291A13DF3
:100D3B00D294D2AF759F00020EB1207D17C2AF7552
:100D4B00430390011CD290306202C291D2AF759FC7
:100D5B0020020EB1C2AF75430390011CD2923062D8
:100D6B0002C291D2AF759F00020EB1D2A0207D11AD
:100D7B00C2AF754304C293D295D2AF759F00020EDA
:100D8B00B1C2AF754304C295D293D2AF759F200207
:100D9B000EB1C2A0307243207D20C2AF75430590C7
:100DAB000130757E08D291C294306204C292A1BD0B
:100DBB00D293D2AF759F10020EB1C2AF754305909F
:100DCB000152757E20D291C294306204C290A1DD93
:100DDB00D295D2AF759F10020EB1207D17C2AF75A1
:100DEB004305900112D291306202C292D2AF759F2D
:100DFB0010020EB1C2AF754305900126D29130623D
:100E0B00EBC290D2AF759F10020EB1D2A0207D1114
:100E1B00C2AF754306C295D294D2AF759F20020E16
:100E2B00B1C2AF754306C293D294D2AF759F000285
:100E3B000EB1C2A0307242207D20C2AF754301902B
:100E4B000152757E20D292C293306204C290C15D72
:100E5B00D295D2AF759F00020EB1C2AF7543019010
:100E6B000130757E08D290C295306204C292C17D6A
:100E7B00D293D2AF759F20C1B1207D16C2AF7543FF
:100E8B0001900126D292306202C290D2AF759F00C0
:100E9B00C1B1C2AF754301900112D290306202C250
:100EAB0092D2AF759F20C26622900110757E00D240
:100EBB0092D291D290C293C294C295C26222788090
:100ECB0076FF0876FF0876FF0876FF08760308762C
:100EDB000408760A087603087601087601788C7682
:100EEB00010876FF0876FF0876FF0876FF0876FF85
:100EFB000876030876FF0876FF0876FF0876250844
:100F0B0076D00876FA0876FA0876040876FF087623
:100F1B000108760008767A0876FF087601087601D4
:100F2B00087600087603227887E6FFC272BF0302B9
:100F3B00D2727888E6C394036008C27DE630E10282
:100F4B00D27DC27E7889E630E102D27EC3EF940275
:100F5B006008758E01D273020F6A758E00C2732200
:100F6B007880E6149000809378A4F67881E614904C
:100F7B0000809378A5F67886E61490008D9378A67A
:100F8B00F6789CE67538FF75390CB402067538A0F7
:100F9B0075390AB4030675388275390578A3E614DA
:100FAB0090009A93F569D1B422227896E6FA789755
:100FBB00E6FB7888E6B40305C3EB940EFB307F04A5
:100FCB007A007BFFC3EB9AFCC3948250027C827540
:100FDB0075000575EC8575F0A4C3E5F0947D40F2C2
:100FEB0022D27FF1B512059C7A007B007C10120592
:100FFB0092E55F2AFA74003BFBDCF37C04C3EB1332
:10100B00FBEA13FADCF7FEC27F120FB522E5EF20E5
:10101B00E6037520000520903FFFE5201460069045
:10102B001DFF1460009304600375EF1253D9BF7555
:10103B0081C043FF8012058D75EF0243B203E5B308
:10104B00240420E70DF521E5E320E0068521B343D9
:10105B00E301120EB47580FF75A40075F1D475D43D
:0D106B00EF75908775A54075F2FF75D5BF34
:1010780075A60175E24275DB4675EA02E4F8F6D812
:10108800FD756B01120EC912155C7898867675305D
:1010980001C2AF1205A61205B612059C1205BD12B3
:1010A800059C1205C412059C1216751205A6120598
:1010B800A61205A1C2AF78FA79FA308407D9FBD80D
:1010C800F7021C00120F32120F6B120FB4120FB579
:1010D80078988676120EB475885075891275C8246A
:1010E80075910475D84075A82275B80275E6907593
:1010F8009B80759D0075D10E75BC5875BB0375BA7C
:101108001175E88012058DD2AF12084653DACF2048
:101118007E0343DA20307E0343DA1043DA01C2D873
:10112800C2711205A6D2617B037A0CE55E70077A5C
:101138000CDB030210BC12059C2070030210BCC219
:1011480070E55FC3940240E1E52F541F856160F5A7
:1011580061B560D5DAD5C26153DACF207E0343DAB0
:1011680020307E0343DA10C2D8C27178A2E6700834
:10117800D274E52F54E0F52FC2757529001205A128
:10118800307409C3E529940A4002D2751205927891
:10119800023074027800C3E55F9840F0C2AF1205D0
:1011A800B61205B61205B6D2AF1205A6754D00786F
:1011B80088E6B40302419C120592788CE6C3940138
:1011C800500302129CE530C39401500302129C2084
:1011D8007435C3E55F94FF500302129CC2AF120539
:1011E800CBD2AF1205A1C3E55F940150EFC2AF1295
:1011F80005B61205971205B6D2AF1205A1C3E55F71
:1012080094FF40E90216FA7F05D27F120FB5120546
:10121800A1C2AFC27F120FB5AE5FC3E55F947FD2A4
:10122800AF407B12058DC2AF1205CBD2AFDFDA1209
:101238000FECC3EE94057897F61205A612159E12C8
:10124800167D7F0AD27F120FB51205A1C2AFC27FE9
:10125800120FB5AE5FC3E55F947FD2AF50E41205BD
:101268008DC2AF1205B61205971205B6D2AFDFD4FC
:10127800120FECEE24057896F61205A612159E12AA
:1012880016AC1205A1120FB5C3E55F94FF500221F9
:10129800D70216FAC3E55F954D4003855F4D1205E9
:1012A800A178017988E7B403027805C3E55F98401F
:1012B8000221B7C2AF1205CB1205CB1205CBD2AFB4
:1012C8001205A6753000E4F531F5320531E531F443
:1012D80070390532789AE6781914601278321460F9
:1012E8000D787D14600878FA146003753200C3E540
:1012F8003298401715327531B478998676C2AF1294
:1013080005CBD2AF789886761205A1120597E52A03
:10131800700530740201BC78012074027806C3E5B8
:101328005F9840A77888E6C3940360031205A1E597
:101338002A70030210BCC2AF120EB4E4F522F523E2
:10134800F524F525F526F56AD2AF7885E6C333F599
:1013580068E4F545F546F547F548F549F573F52C84
:10136800F52DF53775730875BB1012058D12084AEF
:10137800E5E820ECFBA8BDA9BEE97001F888741265
:10138800084E75730875BB107887E6FE7602120F53
:10139800327887EEF6C2AF7564FF1208C6852264FC
:1013A800852265852266D2AF7522017524017525CF
:1013B8000175260185636C756D017888E6B40307AD
:1013C800C27D307602D27DD268D269753300120EA2
:1013D80016120E3D1208E61208ED1208E61208ED84
:1013E8001208E60213FBC2AF120F32D2AF757300B8
:1013F80075BB03120B71120696120C8C120CD612C6
:1014080008ED120B60306D03120697206703120770
:10141800E9306703120830120C8C120CFD1208ED2B
:10142800120B71306D031206D3120C8C120D76124A
:1014380008ED120B60306D03120731120C8C120D7F
:101448009D1208ED120B71306D0312078E120C8C71
:10145800120E161208ED12084A120B60120C8C12AA
:0E1468000E3D12084E1208ED306932206B2F37
:1014760085676485676585636C756D0179187A0C77
:10148600C3E53399400CC269D26A8A357564FF0296
:1014960014A5C3E55F940140030213FB0215223035
:1014A6006A1B206B18E535147004C26A61EEF535C7
:1014B600C3E55F940140030213FB02152275360053
:1014C600C3E5627882985054307404E52A604D78FA
:1014D60088E6B40317207D0520760781F230760270
:1014E60081F2206B07D26B856764813A78F0306BA6
:1014F600058567647820C3E54198500261FB306B2F
:101506001BC26BC27D307602D27DD26A75351285DA
:10151600676461FB0536E55F6002A125753600C28A
:10152600AF120EB47887E6FE7602120F327887EE97
:10153600F6E4F522F523F524F525F526F568C268C7
:10154600D2AF12058D120EB4307409C3E536940578
:10155600400201BC41CE901A0D78201215E0E5201C
:10156600B45A0CA31215E0E520B4A50302157E12A9
:101576000EC912159E02159D901A0378807B0A12D9
:1015860015E0A308DBF9901A0F788C7B181215E08A
:10159600A308DBF9901A2722C2AF12161F1215F9FB
:1015A600901A00740E1215E5A374041215E5A374BF
:1015B600141215E5901A0378807B0A1215E4A30825
:1015C600DBF9901A0F788C7B181215E4A308DBF967
:1015D600121632121610901A2722E493F622E643C8
:1015E6008F01538FFD75EF0275B7A575B7F1F053EF
:1015F6008FFE22438F02438F0175EF0275B7A575E3
:10160600B7F1901A0DF0538FFC22901A0D745AB14F
:10161600E5901A0E74A5B1E5227A3079D07820903B
:101626001A40B1E0E520F709A3DAF7227A3079D03B
:10163600901A40E7B1E509A3DAF922AB77A878BB9F
:1016460001027984BB02027985BB03027986BB0459
:10165600027992BB05027987BB060279A3BB070212
:10166600799CBB08027988BB09027989E8F7227C54
:10167600051205A6DCFB22C2AF1205B61205BD1285
:1016860005C41205CB1205971205B61205BD120543
:10169600C41205CB1205971205B61205BD1205C474
:1016A6001205CBD2AF22C2AF1205CB1205C412056A
:1016B600BD1205B61205971205CB1205C41205BD5B
:1016C6001205B61205971205CB1205C41205BD12F6
:1016D60005B6D2AF22AE77AF78C2AF1205B6120505
:1016E600B61205B6120597DEF21205CB120597DF84
:1016F600F8D2AF22D17DD175D17575770175780194
:10170600757900D1DB7C05AD5F1205A6C3ED955F4B
:1017160070F5C3E55F9401400AC3E55F94FF40326C
:10172600021736D141B19ED17DC2AF75EF12D17588
:10173600DCD50579C3E5799403500280C6D17505D9
:1017460078E5771490009F93F808C3E578985002DF
:1017560080AED175D1750577C3E577940A500280BE
:0D1766009C120EC9B19EC2AF75EF12D17575
:0319FD00021018BD
:101A00000E0414FFFFFFFF03040A0301015AA5019E
:101A1000FFFFFFFFFF03FFFFFF25D0FAFA04FF01DE
:081A2000007AFF01010003FF41
:101A400023484B696E67323041232020202020201C
:101A500023424C48454C4923463333302320202031
:101A60002020202020202020202020202020202076
:101C0000C2AFC2D353D9BF7581C043B20343FF8073
:101C1000752438752503B1C975EF0275E24043F1AB
:101C20001053A4EF75D400D2847DFA780379E67C52
:101C300010752200752300901DD67B0675249875BB
:101C400025013084028142208408D8FBD9F9DCF7D1
:101C500081B4308408D8FBD9F9DCF781B4B189E4C8
:101C600093A3C39A6004DDC381B4DBDBB17B600264
:101C7000812B7B08E493FAA3B15CDBF87A30B15C8A
:101C8000752200752300B17BEAFCEBFDC3ED94FEE9
:101C9000400EB17B8A278B28ED30E0048A828B834B
:101CA000B17B7AC270D8C3ED94FE601350CEBD00F4
:101CB00025EC60097520007521FF0200008100A855
:101CC00027A9280809D804D90281D3B17FEA89AAB3
:101CD000F281C50D81A0C3ED94035049EDA2E092BD
:101CE000007AC5C3E5829400E583941C50902000DF
:101CF00010438F02438F0175B7A575B7F1F030001F
:101D00001FA827A9280809438F01538FFDD804D99C
:101D100002A12089AAE275B7A575B7F1F0A3A10DBC
:101D2000538FFC817C7AC1BD030CE493A3FAB140CC
:101D3000DCF8B138817C817EAA22AB23B15CEBFA5E
:101D4000EA6222752608C3E52313F523E52213F57D
:101D50002250066323A0632201D526EAB1C9B1C986
:101D600075260AEAF4200102D284300102C284B14D
:101D7000C9C3134002C201D526EB22B17FEAFB2082
:101D80008402A17F308402A184752608AE24AF2589
:101D9000C3EF13FFEE13FEB1CDB1C9C3EA13308414
:101DA000024480FA30E703632201C3E52313F523DD
:101DB000E52213F52250066323A0632201D526D91C
:101DC000E52265236523F52222AE24AF250E0FDE22
:101DD000FEDFFCD20122424C48656C693437316326
:041DE000F3300601D5
:00000001FF
